:2000000010CECBEABDF18BCC732110B3CBFE275CFDCBFE7CC83B8ECBEBBDF84FBDF1AFDCDF
:2000200025108301012602D75657C4038EF0FDE685D729C602D724CEFD0DBDF687BDF19298
:20004000BDF289BDF2A9B6C826CEF10C85202702334CBDF3858EF0E9BDF3088603BDF43492
:200060007AC82426F3B6C826810123B0BDF1AF86CC9729CCF101DD390F250F26CE00008E00
:20008000F101C60BA6C0A180270DC1012704C1052305CEE00020075A26EAD739D73A0C5645
:2000A000DF37EEC4BDF1AFCCF848DD2ABDF687BDF192BDF289BDF2A9CCC0C0FEC839BDF303
:2000C0007AB6C83B260C4ACECBEBA746CC68D0BDF37AFEC8373342BDF385B6C85626C5BEAE
:2000E000C8258C000523BD6E4140D60056810000A97E0039DC8E00004A720000B6E0380EA4
:20010000036720474345203139383280F16027CF5645435452455880F36026CF56454354B0
:2001200052455880FC60DFE947434580FC38CCD1454E5445525441494E494E4780FC38BC14
:20014000DC4E455720494445415380008D5CCC9FFFDD02CC0100DD00CC987F970BD704BDDA
:20016000F354203E8D49C67A8EC800BDF53FCCC87DDD7B0C7D27FC86059728CC3075DD3D93
:20018000CC0103DD1FCC0507DD21398DD78DBD7EF272BEC8253001BFC8258D0E8620950D89
:2001A00027FCFCC83DDD087EF2E686D01F8B3986C81F8B39B4C80FB7C80F8EC812A61DA78B
:2001C0001E860E9701CC1901970012D7000F03CC0901970012960143A71DD700C6FFD703CA
:2001E00043AA1E43A71F3402C6011F98A4E4A7805826F735827AC8238EC81FA680260C8C9E
:20020000C82326F76F84860197003997000F010A00C6605C2AFDB6C8232B2586200C0095FA
:2002200000270AC640D7019500260B2008C6C0D701950027015FE71B20C51F989A01970176
:200240008620950026061F989801970154F1C81A26E8D60120E08EC800E7869701861997B2
:2002600000860197009601D701C611D700C601D70039CC0E008DDF4A2AFB7EF5338EC800BB
:2002800020028DD5ECC12AFA398EC800CEC83F860DE6C0E18627028DC04A2AF539861F2028
:2002A0000A863F2006865F2002867F9701B7C827CC05049700D700D700C601D70039F7C84F
:2002C00028EC818D4D86FF970AF6C8285A26FD0F0A397AC8238DEAB6C82326F62076A6807F
:2002E0002E728DDD20F88EF9F08D1DBDF36B8D202062C67FD704A684E60220169701340637
:20030000867F97040F002010C6FF2002C67FD704EC8197010F00340686CE970C0F0A0C008D
:20032000D7010F053506BDF584E77FAA7FC6408140231281642304860820028604D50D2786
:20034000FC4A26FD39D50D27FC39BDF1AA2005B6C8242716CC00CCD70C970ACC03020F0164
:200360009700D700D700C601D70039CC00CCD70C970A39ECC1FDC82AECC1BDF2FCBDF575F1
:200380007EF4958DEEA6C426FA398DECA6C426FA39AE843404C68033783606350281092361
:2003A00002863C8B30C62D3606361020CBA6802008D7042007EC81D704B7C823EC8497011C
:2003C0000F003002120C00D701CC0000201FA6802008D7042007EC81D704B7C823EC84979A
:2003E000010F003002120C00D701CCFF00970AD705CC0040D50D27FC12970AB6C8234A2AA4
:20040000D97EF34FC6FF2006C67F2002E680D704EC0197010F00A68430030C00D701970A3A
:200420000F05CC0040D50D27FC12970AA6842FE07EF34F4AB7C823EC8497010F0030020CAA
:2004400000D701B6C829C640970A0F05F5D00D270B0F0AB6C82326DB39B6C829970A12D53B
:200460000D27F6B6C8230F0A4D26C87EF34FB6C82434027FC824A6802A048DBB20F826057B
:20048000BDF3BC20F14A2705BDF3DD20E93502B7C8247EF34FFFC82C8EF9D4CC18830F0174
:2004A000970B8EF9D4D7000A00CC8081120C00D70097007DC8000C00B6C82B9701CC0100A6
:2004C000FEC82C97002004A686970AA6C02AF8868197000001860197008CFBB4272C308817
:2004E000501F30B3C82CC0025821008681125A26FA9700F6C82AD7010A00CC810112970090
:200500000F01D7009700C603209B8698970B7EF3543414C602200334145FBEC87BA6014989
:20052000494949A802466984690169025A2AEEA6843594C60D8EC83F8D05863FA706394FD5
:2005400020068EC800CC00FF6F8B8300012AF9398680A7855A26FBA78439C6022002C605B4
:200560008EC82E6D8527026A855A2AF739C6032009C6022005C60120015F5A2AFD398EF9D2
:20058000DCA686394D2A044028014A5D2A045028015A393410DD3459C60059495958D73681
:2005A000DC348DE09734D13423080C361E8920024454810922FADD34D6368EFC24E6858EB6
:2005C000FC2CA6869B358B0AC5012604EB8620035AE086D736963635908B108EFC6D5F850A
:2005E000202702C680841F811026015CA68639341096368DE6DD3796368DDEDD393590C0E7
:2006000010D736973B8DE88D544034028D553584B7C836F7C8233408BDF1AF8DD22018B706
:20062000C8363408BDF1AF97238DC4A680A7C02F060F2335880A23A6808D26A7C4A6848D3F
:200640001AABC4A7C0A61F8D12A7C4A6808D12A0C4A7C096232BD426DC3588973BDC3720CF
:2006600004973BDC39D73CC5012704963B200AD63B2A03033C503D8900D63C2A014039E661
:20068000C6E7864A2AF93996562B2827F98EFC8D9F4D86809756ECC1DD4FECC1DD51DF5346
:2006A000BDF533CC1F1FDD5FCC0000DD63DD6597552039CEC85EC602A6C5811F27026CC55B
:2006C0005A2AF59E51CEC85886076CC4A1C42C026FC4E6C0C407E685E7C04C810923EB0AD0
:2006E00057266B96554A2A0286029755E69FC853CEC85E6FC6C54027198EF9E4A6869445BF
:20070000974596558B03A6869A459745C41FD74620238EF9EAA6869445974596558B03A6E9
:20072000869A4597459655488B0333C6C43F589E4DEC85EDC49E53E6809F535D2BA5E6807A
:200740002A06BDF5330F56399F53C43FD757109E4FCEC85E8EC8428602E6C0C501270754C4
:20076000E6A5C40F200754E6A554545454E7864A2AE7CEC8678EC847ECC36D582A0A605803
:20078000E058820060582004EB588900ED818CC84D26E53920C040C0504C4159455280E097
:2007A000C001C02047414D4580FDC84F4D270286015D2702C601FDC879BDF1AFCCF850DD14
:2007C0002A973C2067BDF1924FBDF1B4BDF55ABDF2A9B6C879108EF7948D5AB6C87A108EA3
:2007E000F79F8D51BDF1AF963C2706960F263D0F3C962F279E962E26CC9615269696122760
:200800000F9679270B4C914F230286019779201C967A27B1D61327094C9150230D8601205F
:2008200009D61427A04A26029650977A86F3972F43972E20908EC85E34028D13A6E0270E59
:200840008D1C1F13ECA1BDF37A1F23BDF37839CC2020ED84ED02A704CC3080ED0539CE00D7
:200860000081632308806433C9010020F481092307800A33C81020F533C61F303402340460
:20088000C6054FC1012310C5012704A6E42006A6E044444444840FBBC8237FC823AB8581BE
:2008A0002F2E028B1081392305800A7CC823A7855A2ACF7FC8235FA685813026098620A7CB
:2008C000855CC1052DF13934504FE6802B08E1C027F822014C4C35D08DED81012606A680E0
:2008E000A7C02AFA3934203436EC64ABC4EB41ED642010342034361F30AB64EB6520F0345A
:200900002034361F415F3AA604AB842802867FA1022D15A604A08428028680A1022E095C33
:20092000C10225E21A0120021CFE353635A096672A29847F97678EC8588604BDF6835454EF
:2009400054DA58C407D754D658C438D753D658C407D75DC602D75C867F200D9677276A903F
:200960005B2A055FD777206297774444D653270D9746D6592B0527051F8953D7464481077F
:200980002305810F27014CD65A2B062702880F1F898D37D65D272B965C4A2A028602975C36
:2009A000BDF57E955D27F0D65C58508EC84B3085BDF517840F81052203488B05A784967EB0
:2009C000A701965843944597453996548EC8454D2709301F4424F8E78420F43901020408D8
:2009E00010204080F7EFDF010204FEFDFB0810207F7F80800020505020C8201010402000C7
:200A0000000000083020707010F830F870700060000000707020F070F0F8F87888700888EE
:200A2000808888F8F070F070F88888888888F870807020000020082000000038102044441E
:200A400000FEFFFE0070505078C850202020A820000000084860888830804008888860604B
:200A60001000408888504888488080808820089080D8C88888888888A8888888888808408E
:200A80008008500000700C2070700044107000006C82FFFE007050F8A0105040401070207B
:200AA000000000104820080850F080108888600020782008A888488048808080882008A09E
:200AC00080A8A8888888884020888888505010404008880070A80A2088F860BA382000003A
:200AE0009282FFFE00200050702060004010A8F800700020482070309008F020707800600D
:200B000040001010B888708048E0E098F82008C080A89888F088F020208850A820202040B5
:200B200020080000FE20082088F8F0A238F882389282FFFE000000F87040A8004010A820D2
:200B40004000004048208008F80888408808606020782020B0F8488048808088882008A0A5
:200B60008088888880A8A010208850A85020404010080000FE2078A888F8F0BA7C20444451
:200B80006C82FFFE0000005028989000202000204000008048208088108888808810602082
:200BA000100040008088488848808088882088908888888880909088208820A8882080405D
:200BC000080800004820F070707060446C5038820082FFFE00200050F8986800104000000C
:200BE000800080803070F8701070708070600040000000207888F070F0F88078887070889D
:200C0000F88888F880688870207020508820F870087000F800206020000000388288000092
:200C200000FEFFFE0011413021102031000103060A0F151C242D081008100B08100D0A089E
:200C4000100E0B0908100E0C0A0908100E0D0B0A0908100F0D0C0B0A0908100F0E0C0B0A18
:200C6000090908100F0E0D0C0B0A0909080019324A62798EA2B5C6D5E2EDF5FBFFFFFFFB3E
:200C8000F5EDE2D5C6B5A28E79624A321903BD03870354032402F702CD02A4027E025B028B
:200CA00039021901FB01DE01C301AA0192017C01660152013F012D011C010C00FD00EF0048
:200CC000E200D500C900BE00B300A900A00097008E0086007F00780071006B0065005F0098
:200CE0005A00550050004B00470043003F003C003800350032002F002D002A002800260032
:200D00002400220020001E001C001B0000FEE8FEB6931F0C931F06989F243C1180FD69FD7D
:200D200079210721072107210721072107210E999F240E959B200E21072107210721072192
:200D40000721079DA3280EA0A62B0E220228022D022802220228022D022802220228022DA6
:200D60000228022E022D282180EFFFFEDCBA00000000000000000000000001020100FFFE9E
:200D8000FFFDC3FEB6512450065006500C5006500650045004500450185004500450045007
:200DA0000C500C502450065006500C500650065004500450045018500450045004500C5097
:200DC000182680FDBA9876554433221100000000000000FE28FD79981C103F08981C04989A
:200DE0001C04981C103F08981C04981C04981C08931808981C089C1F08981C089318089863
:200E00001C08931808981C089C1F08981C08931808981C08931808981C089C1F08981C0863
:200E20009318089C1F301A80FFFEDCBA987654321000000000000000FE66FEB60C181118DE
:200E40000C1811180C1811180C120C0611189D21189F2318A12418A326189FA42818071295
:200E60000706003C1880DEEFFEDCBA0000000000000000000000FEB2FEB618061A061C0C66
:200E8000180C1A242318170618061A0C170C18242418A4280CA3260CA1240C9F230C9D21AF
:200EA000189A1F18170618061A0C170C182424241880FFEEDDCC0000000000000000000013
:200EC000000000000000FEE8FEB6969A1D1E9195181E94981B1E8F941814160A8C91151497
:200EE000160A919518321880EEFFFFEEEEDDCCBBAA99888888888888FF16FEB61C061F061B
:200F00001C0618061A06180615061306180613061706181E1880FFFFEEEEDDDDCCCC0000D1
:200F2000000000000000FE28FEB6160F1605160516051A0F160F1D0F1D051D051D05210F51
:200F40001D321D80FE28FEB616061602160216021A0616061D061D021D021D0221061D3235
:200F60001180FE28FEB61B0F160516051605173016051605160517301680FD69FEB6A02339
:200F800012A0230C9C20069E21129C20321380FDC3FEB616041604160416041A081C80A61C
:200FA000A02008BDF3BEB6C880847FB7C8807AC880A6A44784F8E6A05858585857C4F87DB6
:200FC000C8802BDFBDF3DFB6C880850F26E0852027CD394B415252534F465438324C444D13
:200FE0004342434A5438324C444D4342434A00000000CBF2CBF2CBF5CBF8CBFBCBFBF000B9
:20E00000ED77F85030E84D494E4580F85000DE53544F524D80008EC8836F808CCBC526F955
:20E02000BDE8E37CC82486BBB7C8808E0101BFC8818EC8836F808CCB7026F92000BDF1AFED
:20E04000CC0200BDF7A90A790F560F9B8EC8A8BDF84F8EC8AFBDF84F8EC8F9BDF84FCC00D9
:20E0600001BDF87C8EC900BDF84FCC0001BDF87C8EEDAB9FC49FC6860597D997DA97DB2029
:20E0800024BDE866108EC8C4969BAEA63004AFA68EEDA7969BAE86A605840326020CD9CC87
:20E0A0000001BDF87CBDE7E48EC8C4969BAE86A6842B05BDE1292041DCF0830001DDF02761
:20E0C000143408BDF1AABDEACFCEEE2FBDEA9D3508960F27248EC8A8CECBEBBDF8D88EC861
:20E0E000AFCECBEBBDF8D8DCF01026FF44BDF18B0F3B10CECBEA7EF01C3408BDEAF0BDE506
:20E100001EBDE262BDE4B8BDE3533508BDEB43BDEC46BDEC95BDE64725DF96BD1027FF6167
:20E1200096BE1026FF927EE0A59FC2CC7F00DDDC97B78620979C8EE1E79F9D8EC9339FB9C1
:20E14000861D97B80F56CEED77BDF68D3408BDE711BDF6879626850126020AB7BDEAF0BD4C
:20E16000EACFBDF289BDE51EBDF2A5F6C8B7271C8EEF2610BEC8DCBDEA7F8EEF5DBDEA7FA7
:20E180008EEF94BDEA7F35080ADC20C035080F9C860497B7867F97B896B7274AD6B82704BA
:20E1A0000AB82012D626C41F260C4A97B79EC2A686C603BDE9A13408BDEAF0BDF2A9CEEE3F
:20E1C00020BDEA9D108EE0F8CEEDA7B6C89BEEC6BDEAA8BDE51EBDE262BDE4B83508BDEBE8
:20E1E00043BDE64720B2390AB8274E0CEDBDF51784078B04979CDEB98680A7C4DCDC8B084E
:20E20000A7446F45E7466F47BDF5174D2B0C81102C028B0C81602F0E20EE81F02F02800C7F
:20E2200081A02C0220E2A7C8111F891D8A01A7C8106F4231C812109FB939000207100020A8
:20E240001810010005000325075000000100003500000000040408080D0DEE3DEE53EE6FE0
:20E26000EE8E340886C81F8B96BD1026009C96EE102600A79613102600929614273296D48A
:20E2800091D6271C91D8270896D5271496D7262096D78B0C817F221897D796D497D8200E30
:20E2A00096D58B0C817F220897D596D497D60CF296D5270E800297D5D6D6BDE7B5109FCCE3
:20E2C0009FCE96D7270E800297D7D6D8BDE7B5109FD09FD2DCC8D3CCD3D0DDC8DCCAD3CE76
:20E2E000D3D2DDCA961B270F2B040AD420060CD420023408BDE84C86D01F8BBDF2A5C60C63
:20E30000108EC8C88ECB89BDEA8D3588868097EEBDF51784038B0397EF0CF696EE2A190A3A
:20E32000EF270DBDE98A97C80FC9D7CA0FCB358804EE861F97EF3588D6EFC1E02F0C96EF1B
:20E34000800497EF4FBDE94A35880FEF0FEEBDE8373588B6C8E7272B340886C81F8B96E7BB
:20E360002721DCDED3E2DDDE97DCDCE0D3E4DDE097DD3508BDF2A5C60810BEC8DC8EEFB313
:20E38000BDEA7F398EE3A19FA3BDF5178EE4488406AE86EC81DDDC97DE0FDFD7E00FE12039
:20E3A0005896BF2619BDF517847F8B3097A2BDF517843F97E6BDF5178B1097E7204996BD0A
:20E3C00026E3C61CCEC933A6C4270833C8125A26F620340CED0ABF9EDEAF449EE0AF4686EE
:20E3E00040A7C496C026108EE4129F9DBDF517847F8B40979C0CC09EE8A68097A2A68097EE
:20E40000E6A68097E79FE8D6E6BDE7B5109FE29FE439CEC8C4969BEEC6A6C4C603BDE9A1D0
:20E420008EE4269F9D390AC1270686FF979C2017BDF5171F89C4032602CB01CEC8C4969B31
:20E44000EEC6A6C4BDE9A139E450E46AE484E49E7F00282030402830280010301040182033
:20E46000504030283008607F38708000400030201050202840303E701830602018403024AB
:20E48000507F0670007F40106028383028084030287F2018303008684020507F38700080D2
:20E4A0004030603818303020182038402810602000304038507F1C708604CEC90B8EC815BA
:20E4C000B7C88FBDF2A9A6C427226A492719EC45E341ED45EC47E343ED473145BDEA6D335F
:20E4E0004A7AC88F26E0396FC47AC8EAB6C8BD26EEB6C8EE26E9A68427E56F847CC8B66C0A
:20E50000C4FCC8C8ED45FCC8CAED47FCC907ED41FCC909ED438618A7497CC8EA20C1861C80
:20E52000B7C88FCEC933A6C4260933C8127AC88F26F439102B009C8540102600A48520100E
:20E540002600A98510102600D48501102600D8A6418104275685012731B6C8EE262CB6C8B6
:20E56000BD26273408BDF1AF96C8A044D6CAE046BDF593801097838EE23EE643A685D683A6
:20E58000BDE7B510AF48AF4A3508EC44E348ED44EC46E34AED46BDF2A58EE25AA64148AECC
:20E5A000863144E642BDEA8D7EE52AEC44E348291AED44EC46E34A2912ED46BDF2A931440E
:20E5C0008ECBA7C604BDEA8D7EE52A6FC47AC8EB7EE52AA646ABC810A746A1C81126026461
:20E5E000C4BDF2A53144BDEA6D7EE52AA6438103260DA642A1C8102C068B08A742201B649F
:20E60000C4A6C810A7428618A7C810B6C8ED260AB6C8C02605867FB7C8A27EE5966AC8104D
:20E62000260264C47EE5966FC4A64181042715E6435A2710340A86C81F8BA6E4BDE9A1BD38
:20E64000E9A1350A7EE52A3408BDF1AABDF2A9CECB2B860EB7C88FA6C4102700A6E644E1C0
:20E6600041240DCB03E74410AE428EEEBABDEA7F4D102A00837AC8F710270037B6C82684FA
:20E680000126037CC8F8B6C8F8108E7F008EEF04BDE76A108E60808EEF0BBDE76A108E80C0
:20E6A000508EEF15BDE76A108EA0808EEF1CBDE76A20507AC8D97FC8EB7FC8EDB6C87927F6
:20E6C0002BB6C89B448EC8DAF6C8D9E786B6C8DA2605B6C8DB271AB6C89B8B028402B7C8B6
:20E6E0009B448EC8DAE686F7C8D927EBB6C8D9260D8601B7C8BE2006E644E14125056FC4D8
:20E700007AC8EC33457AC88F1026FF4BBDECC920053408BDF1AABDF2A58E8038BFC890B670
:20E72000C8D9271EB7C88F7AC88F2716B6C8918B06B7C891C60410BEC8908EEEEBBDEA7FAA
:20E7400020E53508962684014848488EEEADCECBA7BDF61FD6EC260F96BD2608D6EB2607BD
:20E76000D6ED26031CFE391A013934328EC8C8BDF2F2A6E497041F20BDF312C60CAE61BD1D
:20E78000F40E35B234168ECB2B860EE684270730054A26F7201DA6E484804CA7842A020C80
:20E7A000BDA6E4847FA704A661A701EC62ED020CEC0CF335963436BDF601A7641D58495877
:20E7C000495849ED62E6641D584958495849ED6435B634368DDFEC7C5849ED64EC7A584943
:20E7E000ED6235B686D01F8BBDF27286C81F8B0F9C0F9F0FA20FA58EC90B6F808CCB7126C9
:20E80000F9CC0000DDDEDDE0DDE2DDE497E797BD97BE97EA97EB97EC97F8C640D7F797EDA7
:20E8200097C08E08009FF0860797BF8EE3849FA3CC0000DDC8DDCACC000097D4DDCCDDCE9F
:20E8400097D597D6DDD0DDD297D797D896D48EEEEBCECB89BDF61F867FD6D4BDE7D210BFED
:20E86000C907BFC9093934303408BDF1AABDF272350886A0978F96C8270A2B034A20014CE8
:20E8800097C80FC996CA270A2B034A20014C97CA0FCB96D4270C811F2E034A20014C843FA8
:20E8A00097D4BDE2F28ECB81C608A6848B03A7805A26F73408BDF1AABDEACF5F8620BDE9A9
:20E8C0000BBDE8FD350896C81026FFAA96CA1026FFA496D41026FF9E0A8F1026FF98BDE791
:20E8E000E435B08EEDE0108ECB71CECB81C6088616AFA13008A7C08B0F5A26F539341E8E7F
:20E90000CB8186086C804A26FB2002341E86D01F8B860934026AE42607BDF3543502359E04
:20E92000BDF3548603B7C823A6E44A8ECB81E686C47FE16123DFE0622FDBD7048ECB7148CE
:20E94000AE86BDF2A9BDF2D520CB341E86D01F8B860934026AE42607BDF3543502359EBD5F
:20E96000F3548603B7C8238EC8C8BDF2F2E6E45858EB622FDFC47FD7048ECB71A6E44A488D
:20E98000AE86BDF2A9BDF2D520CA3406BDF517A7E4BDF51781602EF981A02DF5A761350698
:20E9A00039347696ED102700930AEDBDF517841F978B811B2304800420F6C6123DC3C93371
:20E9C0001F03A6C484C0260D0C8B968B811B2FEA0F8B4F20E5A6E4A7418EE2424810AE8629
:20E9E000109F89C620E7C48EE23EA661E686D78B8EE23AE686E7C810A7438EE2524810AE44
:20EA00008610AF4C8EE24A10AE86109F87810626020CF496889B8A19A74F9687998919A731
:20EA20004E968BBDEA3EBDE7B510AF48AF4A0CEB96C0270886FF979C860397C135F63406AF
:20EA4000BDF5171F898430A761C40FC1042402CB04C10C2302C004EB61E761358634068637
:20EA60007F97041F20BDF2C3BDF35435863406867F9704A6A4E622BDF2C3BDF3543586347B
:20EA8000161F20BDF2FCE661BDF40E359634161F21BDF2F2E661AE62BDF40E359634568689
:20EAA0007F9704BDF37335D634561F20BDF2FCBDF49535B6BDF2A9CCFC38FDC82AB6C89B09
:20EAC000108EEDA310AEA6CEED9FEEC68DDA39BDF2A9CCFC38FDC82A108E7FA0CEC8A88D27
:20EAE000C7B6C8792709108E7F10CEC8AF8DB939BDF1923408BDF2E6BDEAB4B6C880BDF11F
:20EB0000B4FCC881FDC81FFDC821BDF1F886C81F8B969C27080A9C2604AD9FC89D969F2756
:20EB2000080A9F2604AD9FC8A096A227080AA22604AD9FC8A396A527080AA52604AD9FC8FB
:20EB4000A6358896EA2712108EC90B8604978F6DA42607312A0A8F26F63996E727353420C3
:20EB6000A625E6271F01CC0616109EDCBDF8FF352024206FA40FE70FA28EED9F969BAE86A5
:20EB8000CC1000BDF87C8630C6709EDCBDE7840AEA20C6CEC933861C9790A6C4843F260911
:20EBA00033C8120A9026F320AA3420A625E6271F01A644E6461F02EC4CBDF8FF352024E003
:20EBC000A6418402275A8EED9F969BAE86EC4EBDF87C0CF5A644E6461F01A642C620BDE7B4
:20EBE00084CC0110ED4E96C8A044D6CAE046BDF59380101F893420863FBDE7B510AF48AFCC
:20EC00004A35206FA4CC0404ED4CA641E6435A2706BDE9A1BDE9A18604A7410AEA7EEB53EE
:20EC20008601A7C46FA48EED9F969BAE86EC4EBDF87CA644E6461F01A642C640BDE7840A8F
:20EC4000EB0AEA7EEB5396BD261996EE2615108EC933861C978FA6A4843F260831A8120A36
:20EC60008F26F339342096C8D6CA1F01A624E62610AE2C1E20BDF8FF352024E06FA40FED27
:20EC800096C8D6CA1F01A6228A80C630BDE7840CF30AEB20CE96BD261996EE261596E7278F
:20ECA0001196C8D6CA1F01CC0616109EDCBDF8FF2501390FE70FA296C8D6CA1F0186088AC3
:20ECC00080C630BDE7840CF339B6C8F227087FC8F2CEED372031B6C8F327087FC8F3CEEDAE
:20ECE0004D2024B6C8B627087FC8B6CEED422017B6C8F4270B7FC8F47FC8F6CEED5A200797
:20ED0000B6C8F626F02003BDF27DF6C800CB10C1A024078600BDF2562006CC0800BDF2566B
:20ED2000F6C802CB20C1F024078602BDF2562006CC0900BDF2563900100100061F0706083B
:20ED40000FFF02390300061F0705090FFF061F07070A100B000C380D00FF00000100023044
:20ED6000030004000500061F073D0800090F0A000B000C000D00FFED8FFEB600190119006E
:20ED8000190132001901190019061905190080FFEEDDCCBBAA99887777777777777777C882
:20EDA000A8C8AF7FA07F10C8F9C900000000000200000001000000030000000201000002F1
:20EDC00003000001030000020200000101000003030000020202000101010003030300808E
:20EDE000C8403F002080101F3F3F00BFBFBFC0204808F830A810D0A0BFBF003F3F482080DE
:20EE000000B04838FB3880283048808045F0287F3FBFA500D0602028B840158040F840185B
:20EE2000FA38E0C84D494E45204649454C4480FA38E0D847414D45204F56455280001000DB
:20EE4000FF20A0FFC040FF9020FF7020FF5050FFD09001002000FF30B0FFB030FFB0D0FF5B
:20EE60003050FFD050FF50D0FF5030FFD0B001FF0000003000FF10C0FFC010FFC0F0FF104A
:20EE800040FFF040FF40F0FF4010FFF0C001FF000000F0D0FFC040FF2000FF4040FF00E09A
:20EEA000FF40C0FFE000FFC0C0FF002001003F00FF8000003F3FFF008001FF7F2000C010AB
:20EEC000FFC0D0FF207F00E0C0FF00C0FFE03000C000FF60CDFFA0000020D0FF3C30FF00B2
:20EEE00082003030FFD050FF20F001003F00FFC408FFD8D8FF2000000040FFE000FF28D80B
:20EF0000FF3C0801003F00FFC40801000408FFD8D8FF200001003F00FFC4F8010004F8FFD1
:20EF2000D828FF200001002000FF00D8FFD0A8FFF040FF0818FF18F0FFF0B8001048FF08E8
:20EF400000FFE810FFF800000800FF00060010FAFF0800FF00F0001018FFF0080100200076
:20EF6000FF0028FFD058FFF0C0FF08E8FF1810FFF0480010B8FF0800FFE8F0FFF800FF08A3
:20EF800000FF00FA001006FF0800FF00100010E8FFF0F801FF00D8FFE808FF0040FF180848
:20EFA000FF00D80008E0FF1000FF0040FFF000FF00C001001800FF0020FFC870FF10A0FF79
:20EFC00000A0FFECA4FF396DFF00200100000000000000000000000000000000000000003D
:20EFE000000000000000000000000000000000000000000000000000000000000000000011
:20F00000ED77F85030E84D494E4580F85000DE53544F524D80008EC8836F808CCBC526F945
:20F02000BDE8E37CC82486BBB7C8808E0101BFC8818EC8836F808CCB7026F92000BDF1AFDD
:20F04000CC0200BDF7A90A790F560F9B8EC8A8BDF84F8EC8AFBDF84F8EC8F9BDF84FCC00C9
:20F0600001BDF87C8EC900BDF84FCC0001BDF87C8EEDAB9FC49FC6860597D997DA97DB2019
:20F0800024BDE866108EC8C4969BAEA63004AFA68EEDA7969BAE86A605840326020CD9CC77
:20F0A0000001BDF87CBDE7E48EC8C4969BAE86A6842B05BDE1292041DCF0830001DDF02751
:20F0C000143408BDF1AABDEACFCEEE2FBDEA9D3508960F27248EC8A8CECBEBBDF8D88EC851
:20F0E000AFCECBEBBDF8D8DCF01026FF44BDF18B0F3B10CECBEA7EF01C3408BDEAF0BDE5F6
:20F100001EBDE262BDE4B8BDE3533508BDEB43BDEC46BDEC95BDE64725DF96BD1027FF6157
:20F1200096BE1026FF927EE0A59FC2CC7F00DDDC97B78620979C8EE1E79F9D8EC9339FB9B1
:20F14000861D97B80F56CEED77BDF68D3408BDE711BDF6879626850126020AB7BDEAF0BD3C
:20F16000EACFBDF289BDE51EBDF2A5F6C8B7271C8EEF2610BEC8DCBDEA7F8EEF5DBDEA7F97
:20F180008EEF94BDEA7F35080ADC20C035080F9C860497B7867F97B896B7274AD6B82704AA
:20F1A0000AB82012D626C41F260C4A97B79EC2A686C603BDE9A13408BDEAF0BDF2A9CEEE2F
:20F1C00020BDEA9D108EE0F8CEEDA7B6C89BEEC6BDEAA8BDE51EBDE262BDE4B83508BDEBD8
:20F1E00043BDE64720B2390AB8274E0CEDBDF51784078B04979CDEB98680A7C4DCDC8B083E
:20F20000A7446F45E7466F47BDF5174D2B0C81102C028B0C81602F0E20EE81F02F02800C6F
:20F2200081A02C0220E2A7C8111F891D8A01A7C8106F4231C812109FB93900020710002098
:20F240001810010005000325075000000100003500000000040408080D0DEE3DEE53EE6FD0
:20F26000EE8E340886C81F8B96BD1026009C96EE102600A79613102600929614273296D47A
:20F2800091D6271C91D8270896D5271496D7262096D78B0C817F221897D796D497D8200E20
:20F2A00096D58B0C817F220897D596D497D60CF296D5270E800297D5D6D6BDE7B5109FCCD3
:20F2C0009FCE96D7270E800297D7D6D8BDE7B5109FD09FD2DCC8D3CCD3D0DDC8DCCAD3CE66
:20F2E000D3D2DDCA961B270F2B040AD420060CD420023408BDE84C86D01F8BBDF2A5C60C53
:20F30000108EC8C88ECB89BDEA8D3588868097EEBDF51784038B0397EF0CF696EE2A190A2A
:20F32000EF270DBDE98A97C80FC9D7CA0FCB358804EE861F97EF3588D6EFC1E02F0C96EF0B
:20F34000800497EF4FBDE94A35880FEF0FEEBDE8373588B6C8E7272B340886C81F8B96E7AB
:20F360002721DCDED3E2DDDE97DCDCE0D3E4DDE097DD3508BDF2A5C60810BEC8DC8EEFB303
:20F38000BDEA7F398EE3A19FA3BDF5178EE4488406AE86EC81DDDC97DE0FDFD7E00FE12029
:20F3A0005896BF2619BDF517847F8B3097A2BDF517843F97E6BDF5178B1097E7204996BDFA
:20F3C00026E3C61CCEC933A6C4270833C8125A26F620340CED0ABF9EDEAF449EE0AF4686DE
:20F3E00040A7C496C026108EE4129F9DBDF517847F8B40979C0CC09EE8A68097A2A68097DE
:20F40000E6A68097E79FE8D6E6BDE7B5109FE29FE439CEC8C4969BEEC6A6C4C603BDE9A1C0
:20F420008EE4269F9D390AC1270686FF979C2017BDF5171F89C4032602CB01CEC8C4969B21
:20F44000EEC6A6C4BDE9A139E450E46AE484E49E7F00282030402830280010301040182023
:20F46000504030283008607F38708000400030201050202840303E7018306020184030249B
:20F48000507F0670007F40106028383028084030287F2018303008684020507F38700080C2
:20F4A0004030603818303020182038402810602000304038507F1C708604CEC90B8EC815AA
:20F4C000B7C88FBDF2A9A6C427226A492719EC45E341ED45EC47E343ED473145BDEA6D334F
:20F4E0004A7AC88F26E0396FC47AC8EAB6C8BD26EEB6C8EE26E9A68427E56F847CC8B66CFA
:20F50000C4FCC8C8ED45FCC8CAED47FCC907ED41FCC909ED438618A7497CC8EA20C1861C70
:20F52000B7C88FCEC933A6C4260933C8127AC88F26F439102B009C8540102600A4852010FE
:20F540002600A98510102600D48501102600D8A6418104275685012731B6C8EE262CB6C8A6
:20F56000BD26273408BDF1AF96C8A044D6CAE046BDF593801097838EE23EE643A685D68396
:20F58000BDE7B510AF48AF4A3508EC44E348ED44EC46E34AED46BDF2A58EE25AA64148AEBC
:20F5A000863144E642BDEA8D7EE52AEC44E348291AED44EC46E34A2912ED46BDF2A93144FE
:20F5C0008ECBA7C604BDEA8D7EE52A6FC47AC8EB7EE52AA646ABC810A746A1C81126026451
:20F5E000C4BDF2A53144BDEA6D7EE52AA6438103260DA642A1C8102C068B08A742201B648F
:20F60000C4A6C810A7428618A7C810B6C8ED260AB6C8C02605867FB7C8A27EE5966AC8103D
:20F62000260264C47EE5966FC4A64181042715E6435A2710340A86C81F8BA6E4BDE9A1BD28
:20F64000E9A1350A7EE52A3408BDF1AABDF2A9CECB2B860EB7C88FA6C4102700A6E644E1B0
:20F6600041240DCB03E74410AE428EEEBABDEA7F4D102A00837AC8F710270037B6C82684EA
:20F680000126037CC8F8B6C8F8108E7F008EEF04BDE76A108E60808EEF0BBDE76A108E80B0
:20F6A000508EEF15BDE76A108EA0808EEF1CBDE76A20507AC8D97FC8EB7FC8EDB6C87927E6
:20F6C0002BB6C89B448EC8DAF6C8D9E786B6C8DA2605B6C8DB271AB6C89B8B028402B7C8A6
:20F6E0009B448EC8DAE686F7C8D927EBB6C8D9260D8601B7C8BE2006E644E14125056FC4C8
:20F700007AC8EC33457AC88F1026FF4BBDECC920053408BDF1AABDF2A58E8038BFC890B660
:20F72000C8D9271EB7C88F7AC88F2716B6C8918B06B7C891C60410BEC8908EEEEBBDEA7F9A
:20F7400020E53508962684014848488EEEADCECBA7BDF61FD6EC260F96BD2608D6EB2607AD
:20F76000D6ED26031CFE391A013934328EC8C8BDF2F2A6E497041F20BDF312C60CAE61BD0D
:20F78000F40E35B234168ECB2B860EE684270730054A26F7201DA6E484804CA7842A020C70
:20F7A000BDA6E4847FA704A661A701EC62ED020CEC0CF335963436BDF601A7641D58495867
:20F7C000495849ED62E6641D584958495849ED6435B634368DDFEC7C5849ED64EC7A584933
:20F7E000ED6235B686D01F8BBDF27286C81F8B0F9C0F9F0FA20FA58EC90B6F808CCB7126B9
:20F80000F9CC0000DDDEDDE0DDE2DDE497E797BD97BE97EA97EB97EC97F8C640D7F797ED97
:20F8200097C08E08009FF0860797BF8EE3849FA3CC0000DDC8DDCACC000097D4DDCCDDCE8F
:20F8400097D597D6DDD0DDD297D797D896D48EEEEBCECB89BDF61F867FD6D4BDE7D210BFDD
:20F86000C907BFC9093934303408BDF1AABDF272350886A0978F96C8270A2B034A20014CD8
:20F8800097C80FC996CA270A2B034A20014C97CA0FCB96D4270C811F2E034A20014C843F98
:20F8A00097D4BDE2F28ECB81C608A6848B03A7805A26F73408BDF1AABDEACF5F8620BDE999
:20F8C0000BBDE8FD350896C81026FFAA96CA1026FFA496D41026FF9E0A8F1026FF98BDE781
:20F8E000E435B08EEDE0108ECB71CECB81C6088616AFA13008A7C08B0F5A26F539341E8E6F
:20F90000CB8186086C804A26FB2002341E86D01F8B860934026AE42607BDF3543502359EF4
:20F92000BDF3548603B7C823A6E44A8ECB81E686C47FE16123DFE0622FDBD7048ECB7148BE
:20F94000AE86BDF2A9BDF2D520CB341E86D01F8B860934026AE42607BDF3543502359EBD4F
:20F96000F3548603B7C8238EC8C8BDF2F2E6E45858EB622FDFC47FD7048ECB71A6E44A487D
:20F98000AE86BDF2A9BDF2D520CA3406BDF517A7E4BDF51781602EF981A02DF5A761350688
:20F9A00039347696ED102700930AEDBDF517841F978B811B2304800420F6C6123DC3C93361
:20F9C0001F03A6C484C0260D0C8B968B811B2FEA0F8B4F20E5A6E4A7418EE2424810AE8619
:20F9E000109F89C620E7C48EE23EA661E686D78B8EE23AE686E7C810A7438EE2524810AE34
:20FA00008610AF4C8EE24A10AE86109F87810626020CF496889B8A19A74F9687998919A721
:20FA20004E968BBDEA3EBDE7B510AF48AF4A0CEB96C0270886FF979C860397C135F634069F
:20FA4000BDF5171F898430A761C40FC1042402CB04C10C2302C004EB61E761358634068627
:20FA60007F97041F20BDF2C3BDF35435863406867F9704A6A4E622BDF2C3BDF3543586346B
:20FA8000161F20BDF2FCE661BDF40E359634161F21BDF2F2E661AE62BDF40E359634568679
:20FAA0007F9704BDF37335D634561F20BDF2FCBDF49535B6BDF2A9CCFC38FDC82AB6C89BF9
:20FAC000108EEDA310AEA6CEED9FEEC68DDA39BDF2A9CCFC38FDC82A108E7FA0CEC8A88D17
:20FAE000C7B6C8792709108E7F10CEC8AF8DB939BDF1923408BDF2E6BDEAB4B6C880BDF10F
:20FB0000B4FCC881FDC81FFDC821BDF1F886C81F8B969C27080A9C2604AD9FC89D969F2746
:20FB2000080A9F2604AD9FC8A096A227080AA22604AD9FC8A396A527080AA52604AD9FC8EB
:20FB4000A6358896EA2712108EC90B8604978F6DA42607312A0A8F26F63996E727353420B3
:20FB6000A625E6271F01CC0616109EDCBDF8FF352024206FA40FE70FA28EED9F969BAE8695
:20FB8000CC1000BDF87C8630C6709EDCBDE7840AEA20C6CEC933861C9790A6C4843F260901
:20FBA00033C8120A9026F320AA3420A625E6271F01A644E6461F02EC4CBDF8FF352024E0F3
:20FBC000A6418402275A8EED9F969BAE86EC4EBDF87C0CF5A644E6461F01A642C620BDE7A4
:20FBE00084CC0110ED4E96C8A044D6CAE046BDF59380101F893420863FBDE7B510AF48AFBC
:20FC00004A35206FA4CC0404ED4CA641E6435A2706BDE9A1BDE9A18604A7410AEA7EEB53DE
:20FC20008601A7C46FA48EED9F969BAE86EC4EBDF87CA644E6461F01A642C640BDE7840A7F
:20FC4000EB0AEA7EEB5396BD261996EE2615108EC933861C978FA6A4843F260831A8120A26
:20FC60008F26F339342096C8D6CA1F01A624E62610AE2C1E20BDF8FF352024E06FA40FED17
:20FC800096C8D6CA1F01A6228A80C630BDE7840CF30AEB20CE96BD261996EE261596E7277F
:20FCA0001196C8D6CA1F01CC0616109EDCBDF8FF2501390FE70FA296C8D6CA1F0186088AB3
:20FCC00080C630BDE7840CF339B6C8F227087FC8F2CEED372031B6C8F327087FC8F3CEED9E
:20FCE0004D2024B6C8B627087FC8B6CEED422017B6C8F4270B7FC8F47FC8F6CEED5A200787
:20FD0000B6C8F626F02003BDF27DF6C800CB10C1A024078600BDF2562006CC0800BDF2565B
:20FD2000F6C802CB20C1F024078602BDF2562006CC0900BDF2563900100100061F0706082B
:20FD40000FFF02390300061F0705090FFF061F07070A100B000C380D00FF00000100023034
:20FD6000030004000500061F073D0800090F0A000B000C000D00FFED8FFEB600190119005E
:20FD8000190132001901190019061905190080FFEEDDCCBBAA99887777777777777777C872
:20FDA000A8C8AF7FA07F10C8F9C900000000000200000001000000030000000201000002E1
:20FDC00003000001030000020200000101000003030000020202000101010003030300807E
:20FDE000C8403F002080101F3F3F00BFBFBFC0204808F830A810D0A0BFBF003F3F482080CE
:20FE000000B04838FB3880283048808045F0287F3FBFA500D0602028B840158040F840184B
:20FE2000FA38E0C84D494E45204649454C4480FA38E0D847414D45204F56455280001000CB
:20FE4000FF20A0FFC040FF9020FF7020FF5050FFD09001002000FF30B0FFB030FFB0D0FF4B
:20FE60003050FFD050FF50D0FF5030FFD0B001FF0000003000FF10C0FFC010FFC0F0FF103A
:20FE800040FFF040FF40F0FF4010FFF0C001FF000000F0D0FFC040FF2000FF4040FF00E08A
:20FEA000FF40C0FFE000FFC0C0FF002001003F00FF8000003F3FFF008001FF7F2000C0109B
:20FEC000FFC0D0FF207F00E0C0FF00C0FFE03000C000FF60CDFFA0000020D0FF3C30FF00A2
:20FEE00082003030FFD050FF20F001003F00FFC408FFD8D8FF2000000040FFE000FF28D8FB
:20FF0000FF3C0801003F00FFC40801000408FFD8D8FF200001003F00FFC4F8010004F8FFC1
:20FF2000D828FF200001002000FF00D8FFD0A8FFF040FF0818FF18F0FFF0B8001048FF08D8
:20FF400000FFE810FFF800000800FF00060010FAFF0800FF00F0001018FFF0080100200066
:20FF6000FF0028FFD058FFF0C0FF08E8FF1810FFF0480010B8FF0800FFE8F0FFF800FF0893
:20FF800000FF00FA001006FF0800FF00100010E8FFF0F801FF00D8FFE808FF0040FF180838
:20FFA000FF00D80008E0FF1000FF0040FFF000FF00C001001800FF0020FFC870FF10A0FF69
:20FFC00000A0FFECA4FF396DFF00200100000000000000000000000000000000000000002D
:20FFE000000000000000000000000000000000000000000000000000000000000000000001
:00000001FF
